:020000040000FA
:0200000077285F
:0800080009009801831603139F
:1000100098010C30990024309800C0308B008C1669
:10002000831203138030980008004130322054308E
:1000300032202B30322049303220503032205230A2
:1000400032203D30322031303220393032203230CF
:10005000322030303220303032200D3032200A3021
:10006000322008000C1E3228990008000D30322082
:100070000A303220080041303220543032202B30F8
:100080003220433032204D30322053303220533032
:1000900032203D30322008003B20313032203620E3
:1000A00008003B2032303220362008003B2033301D
:1000B0003220362008004130322054303220443083
:1000C00032203E303220533032204D303220313019
:1000D00032203B3032200D303220080041303220B7
:1000E00054303220483032200D30322008008B133B
:1000F0008312850107309F0000308316850083122C
:100100008601FB30831686008312C901861E882A69
:10011000061E2A2A831679309B001C1483120310B2
:100120001A1802299A18C528A22883121C221C22F8
:1001300005118511C910003083169A0079309B0093
:1001400078220E228312061E2A2A861E882A392128
:10015000C91CA228AB288312052064001520023098
:1001600083169A0079309B0078228312C910851576
:100170000E228511061FC0283921C91CBA289528CE
:100180000510851085151C22051183128515640044
:10019000FF306200C910061BD1283921C9189528E3
:1001A000C7284C206400FF3062000130BD000515F7
:1001B0008511C421C91CDD2895288515C421C91CB9
:1001C000E2289528BC0BD728BD0BD7280511061BA4
:1001D000EA28FC285620851505150E220E228511C9
:1001E00005113921C91CF52895280E220E220E2250
:1001F0000E22061BEB28FC28013083169A0079306A
:100200009B00782283126400FF306200851505117F
:10021000061F0F290B29C421C91C0F2995288511F8
:10022000061F17291329C421C91C0229952851200A
:100230006400FF306200061BD128C421C91C252997
:10024000C91C2529C91C2529952885116400FF3062
:100250006200061BD128C421C91C2F299528C4215E
:10026000C91C33299528C421C91C3729952885150F
:1002700018290A22E3210422D5210A22F821061C8A
:100280004E29F121061C45294E29E321061C4E2941
:1002900050216F21A422491D4E29922104220800D9
:1002A0003330B6000830BA000422361C58295A29C7
:1002B000F1216929000000000000000000000A226E
:1002C000F1216A2900000000000000000000000089
:1002D00054290A22B60CBA0B6229F1210800031036
:1002E000203084000830BA0083169B0183127E21DF
:1002F00035088000840ABA0B772908000830BB0053
:10030000042200000000000000000A22F821061C60
:100310008B29B5178C29B513B50CF121BB0B80299E
:10032000B50D0800C801A1290830C8077830480277
:10033000031DA129C9100422E32105150E22051170
:10034000080020308400480883169B008312083080
:10035000BA0083161C148312031083161A08831222
:100360000002031D9429840A83169B0A8312BA0B88
:10037000A9290030A000A100A200A300A400A500AC
:10038000A600A700C91408006400FF306200B00195
:10039000B101A030B200B00BCE29D2293921C91C3D
:1003A000D2290800B20BCB2908000630B100B000FA
:1003B000B00BD829B10BD7290730B100B000B00B72
:1003C000DF29B10BDE290430B100B000B00BE62903
:1003D000B10BE5290530B100B000B00BED29B10B30
:1003E000EC290430B100B000B00BF429B10BF329B3
:1003F00000000000000000000000000000000000FD
:100400006400FF3062000800061083160610831295
:10041000061008008316061483120800B001B1010B
:100420000530B200B00B122AB10B122A6400FF3063
:100430006200B20B122A0800B001B1010130B20013
:10044000B00B202A6400FF306200B10B202AB20BEF
:10045000202A0800BC01BD01061E2A2A2F2ABD0B36
:10046000382ABC0B382A05151C2205118511A22833
:10047000851549110A22F1210422D5210A22F821E9
:10048000061C2F2AF121061C462A2F2AE321061CCE
:100490002F2A50216F21A422491D2F2A4F2A83166B
:1004A00078309B001C141A02031D572A9A018316E8
:1004B0001A089B0083120830BA002030840000081C
:1004C00083169A0078228312840A83169B0A831269
:1004D000BA0B5F2A83161B089A0078309B008312A0
:1004E000782205151C22051185111C2285152A2A42
:1004F00083161C151C108B1355309D00AA309D00CF
:100500009C141C1183128C1F832A8C1383120800E5
:100510008312003083169B0008309A0083127830D3
:10052000BA00782283169B0A8312BA0B912A05150A
:1005300085151C22051185110E22783083169B002B
:1005400000309A0078222A2ABE0149112008C100F1
:10055000C3222108C100C3222208C100C3222308EC
:10056000C100C3222408C100C3222508C100C32240
:100570002608C100C3222708C100C32200303E0262
:100580000319491508000830C00041083E06BF00A5
:100590003F0C3E080318183ABF003F0CBE00031082
:0A05A000C10C4108C00BC62A080078
:02400E000D3F64
:00000001FF
